:100000000C9462000C948A000C948A000C948A0070
:100010000C948A000C948A000C948A000C948A0038
:100020000C948A000C948A000C948A000C948A0028
:100030000C948A000C948A000C948A000C948A0018
:100040000C94EB000C948A000C94DA010C948A0056
:100050000C948A000C948A000C948A000C948A00F8
:100060000C948A000C948A000000000024002700F1
:100070002A0000000000250028002B0000000000DE
:1000800023002600290004040404040404040202DA
:100090000202020203030303030301020408102007
:1000A0004080010204081020010204081020000012
:1000B0000007000201000003040600000000000029
:1000C00000005F0311241FBECFEFD8E0DEBFCDBF1D
:1000D00011E0A0E0B1E0E2EBFAE002C005900D9281
:1000E000A431B107D9F711E0A4E1B1E001C01D923C
:1000F000A63BB107E1F710E0C4ECD0E004C02297C2
:10010000FE010E945305C23CD107C9F70E94E400DA
:100110000C9457050C94000083EA91E00E941003B0
:10012000882371F183EA91E00E94240390931501E2
:10013000809314018930910579F483EA91E049E0D4
:1001400050E060E070E020E030E00E94B9048AE016
:1001500061E00E948D0108958A30910511F00097A9
:1001600079F4AC01662757FD6095762F83EA91E01C
:1001700020E030E00E94B9048AE060E00E948D0136
:1001800008950F931F9303EA11E0C80140E05BE478
:1001900060E070E00E941702C80160E071E00E9418
:1001A000EF038AE061E00E946D018DE061E00E9452
:1001B0006D018AE060E00E948D018DE061E00E94A7
:1001C0008D011F910F9108950E9433010E94C1007B
:1001D0000E948C00FDCF1F920F920FB60F92112438
:1001E0002F933F938F939F93AF93BF9380911A0167
:1001F00090911B01A0911C01B0911D0130911E0135
:100200000196A11DB11D232F2D5F2D3720F02D57F5
:100210000196A11DB11D20931E0180931A01909398
:100220001B01A0931C01B0931D01809116019091B8
:100230001701A0911801B09119010196A11DB11DDE
:100240008093160190931701A0931801B0931901A0
:10025000BF91AF919F918F913F912F910F900FBEC2
:100260000F901F901895789484B5826084BD84B5F2
:10027000816084BD85B5826085BD85B5816085BDA1
:10028000EEE6F0E0808181608083E1E8F0E080814B
:1002900082608083808181608083E0E8F0E08081FB
:1002A00081608083E1EBF0E0808184608083E0EB1B
:1002B000F0E0808181608083EAE7F0E08081846003
:1002C000808380818260808380818160808380815F
:1002D000806880831092C1000895282F30E0C90102
:1002E00086569F4FFC0194912A573F4FF901849104
:1002F000882391F0E82FF0E0EE0FFF1FE859FF4F41
:10030000A591B491662329F48C91909589238C93BF
:1003100008958C91892B8C930895482F50E0CA0141
:1003200082559F4FFC012491CA0186569F4FFC01C4
:1003300094914A575F4FFA0134913323D1F122232C
:1003400031F1233021F4809180008F7705C0243073
:1003500031F4809180008F7D8093800018C021301F
:1003600019F484B58F7704C0223021F484B58F7DD1
:1003700084BD0DC0263021F48091B0008F7705C078
:10038000273029F48091B0008F7D8093B000E32F57
:10039000F0E0EE0FFF1FEE58FF4FA591B4916623DA
:1003A00029F48C91909589238C9308958C91892BB5
:1003B0008C9308951F920F920FB60F9211242F93D2
:1003C0003F934F935F936F937F938F939F93AF93DD
:1003D000BF93EF93FF934091C600E0919F01F0918E
:1003E000A001CF01019660E870E00E94ED049C013D
:1003F0008091A1019091A2012817390739F0E15E9F
:10040000FE4F40833093A00120939F01FF91EF9115
:10041000BF91AF919F918F917F916F915F914F911C
:100420003F912F910F900FBE0F901F9018955F92E4
:100430006F927F928F929F92AF92BF92CF92DF92F4
:10044000EF92FF920F931F93CF93DF93EC013A014A
:100450004B01413482E458078FE0680780E0780759
:100460000CF07FC060E874E88EE190E0A401930195
:100470000E9422052150304040405040CA01B9013D
:1004800022E030E040E050E00E94220559016A017C
:10049000A6019501209530954095509594E0220F46
:1004A000331F441F551F9A95D1F760E074E284EF23
:1004B00090E00E942205CA01B9012FEF30E040E030
:1004C00050E00E94CE04A40193010E942205C901BC
:1004D00081509F4F181619061CF4522E5A9403C0CF
:1004E00055245394521A60E079E08DE390E0A40122
:1004F00093010E9422052150304040405040CA01E3
:10050000B90122E030E040E050E00E942205209551
:1005100030954095509583E0220F331F441F551F9F
:100520008A95D1F760E074E284EF90E00E942205A2
:10053000CA01B9012FEF30E040E050E00E94CE0444
:10054000A40193010E942205C90181509F4F1816F2
:1005500019061CF4822F815002C081E0821B851590
:1005600000F5E885F98581E090E00A8802C0880FEF
:10057000991F0A94E2F7808360E079E08DE390E0D0
:10058000A40193010E942205215030404040504078
:10059000CA01B90122E030E040E050E00E942205AB
:1005A00004C0E885F98510829501EC81FD813083D6
:1005B000EE81FF812083EA85FB85208141E050E0C8
:1005C000CA010E8402C0880F991F0A94E2F7282BF3
:1005D0002083EA85FB852081CA010F8402C0880F31
:1005E000991F0A94E2F7282B2083EA85FB858081F6
:1005F000088802C0440F551F0A94E2F7842B8083B9
:10060000DF91CF911F910F91FF90EF90DF90CF90EE
:10061000BF90AF909F908F907F906F905F90089564
:10062000DC011296ED91FC911397E058FF4F8191F8
:10063000919180589F4F20813181821B930B60E8FC
:1006400070E00E94ED040895CF93DF93DC011296D1
:10065000ED91FC911397EF01CE57DF4F48815981FF
:10066000E058FF4F80819181E058F0408417950752
:1006700019F42FEF3FEF0CC0E40FF51F2081CA01E2
:10068000019660E870E00E94ED049983888330E071
:10069000C901DF91CF910895FC01A085B185218921
:1006A0008C9190E0022E02C0959587950A94E2F70E
:1006B00080FFF6CF0484F585E02D608308958EE0F9
:1006C00091E09093A4018093A3018FE191E0909336
:1006D000A6018093A50185EC90E09093A8018093FA
:1006E000A70184EC90E09093AA018093A90180EC8B
:1006F00090E09093AC018093AB0181EC90E09093FB
:10070000AE018093AD0186EC90E09093B0018093B0
:10071000AF0184E08093B10183E08093B20187E070
:100720008093B30185E08093B40181E08093B501AB
:1007300008950F931F93CF93DF938C01EB0109C0B2
:100740002196D801ED91FC910190F081E02DC80136
:10075000099568816623A1F7DF91CF911F910F91D1
:100760000895EF92FF920F931F93CF93DF938C0125
:100770007B01EA010CC0D7016D917D01D801ED919B
:10078000FC910190F081E02DC801099521972097F7
:1007900091F7DF91CF911F910F91FF90EF90089506
:1007A000DC01ED91FC910280F381E02D0995089523
:1007B0000F931F938C01DC01ED91FC910190F0816E
:1007C000E02D6DE00995D801ED91FC910190F0814B
:1007D000E02DC8016AE009951F910F9108950F93CC
:1007E0001F938C010E94D003C8010E94D8031F915F
:1007F0000F9108952F923F924F925F926F927F9246
:100800008F929F92AF92BF92CF92DF92EF92FF9220
:100810000F931F93DF93CF93CDB7DEB7A0970FB69B
:10082000F894DEBF0FBECDBF1C016A017B014115EC
:1008300051056105710549F4DC01ED91FC910190D0
:10084000F081E02D60E3099554C088249924540177
:10085000422E55246624772401E010E00C0F1D1F62
:10086000080D191DC701B601A30192010E940005E0
:10087000F80160830894811C911CA11CB11CC70164
:10088000B601A30192010E940005C901DA016C01C1
:100890007D01C114D104E104F104F1F681E0E82EF8
:1008A000F12CEC0EFD1EE80CF91C3E010894611CB5
:1008B000711CD501C4010197A109B1096C01C818C7
:1008C000D90814C0F601EE0DFF1D60816A3010F4E6
:1008D000605D01C0695CD101ED91FC910190F081F6
:1008E000E02DC10109950894E108F1086E147F0418
:1008F00049F7A0960FB6F894DEBF0FBECDBFCF91DB
:10090000DF911F910F91FF90EF90DF90CF90BF90FC
:10091000AF909F908F907F906F905F904F903F909F
:100920002F900895EF92FF920F931F93CF93DF9331
:10093000EC017A018B0177FF0FC0E881F98101900A
:10094000F081E02D6DE2099510950095F094E0940A
:10095000E11CF11C011D111DCE01B801A7012AE007
:100960000E94FA03DF91CF911F910F91FF90EF90BA
:100970000895DC012115310541F4ED91FC910190C0
:10098000F081E02D642F099508952A30310519F47E
:100990000E94920408950E94FA030895629FD00174
:1009A000739FF001829FE00DF11D649FE00DF11D2A
:1009B000929FF00D839FF00D749FF00D659FF00DD9
:1009C0009927729FB00DE11DF91F639FB00DE11DC6
:1009D000F91FBD01CF011124089597FB092E0726A9
:1009E0000AD077FD04D049D006D000201AF47095C3
:1009F00061957F4F0895F6F7909581959F4F0895E3
:100A0000A1E21A2EAA1BBB1BFD010DC0AA1FBB1F12
:100A1000EE1FFF1FA217B307E407F50720F0A21B84
:100A2000B30BE40BF50B661F771F881F991F1A94F1
:100A300069F760957095809590959B01AC01BD011B
:100A4000CF01089597FB092E05260ED057FD04D03F
:100A5000D7DF0AD0001C38F4509540953095219589
:100A60003F4F4F4F5F4F0895F6F7909580957095E3
:100A700061957F4F8F4F9F4F0895AA1BBB1B51E17C
:100A800007C0AA1FBB1FA617B70710F0A61BB70BFE
:100A9000881F991F5A95A9F780959095BC01CD01A3
:100AA0000895EE0FFF1F0590F491E02D0994F8943E
:020AB000FFCF76
:100AB200456D70657A616D6F7300000000004C0334
:040AC2009903B103E0
:00000001FF
